:1000000010C02AC028C027C026C025C024C023C0D5
:1000100022C021C00000C037D85D884C094D288C13
:10002000040011241FBECFE9CDBF10E0A0E6B0E070
:10003000E6E4F3E003C0C89531960D92A036B1070F
:10004000D1F710E0A0E6B0E001C01D92A036B107E4
:10005000E1F7D0D077C1D4CF1F920F920FB60F9295
:1000600011242F938F939F9312BE2AEF92B782B7DA
:100070009817E9F3B19905C082B78B3FB8F322BF57
:10008000F5CF9F918F912F910F900FBE0F901F90E2
:100090001895BB98C39ABC98C49AC398BB9A089504
:1000A000C498BC9A90E087FF03C0BB98C39A02C073
:1000B000C398BB9ABC98C49AB49BFECF880FC498CF
:1000C000BC9A9F5F98307CF3BB98C39AC498BC9A43
:1000D000BC98C49A0000C498BC9A0895C398BB9A6F
:1000E0000000BC98C49A0000BB98C39A0895E19997
:1000F000FECF8EBB81E08CBB8DB399270895EF9224
:10010000FF920F931F93082F1127000F111F802FAD
:10011000885FEDDFE82EFF24802F875FE8DF9927D7
:10012000982F88278E299F291F910F91FF90EF907C
:100130000895DF92EF92FF920F931F93CF9324E2E3
:10014000883B920710F4CCE407C0A7E280319A07FD
:1001500010F4CBE401C0CAE4AA27BB2720E137E2B0
:1001600040E050E0682F792F8A2F9B2FD0D0E62EC9
:10017000F72E082F192F88E297E4AAEFBFEFE80EB9
:10018000F91E0A1F1B1F5DE016950795F794E7946B
:100190005A95D1F7BB27A12F902F8F2D30ECD32E5E
:1001A000D82A77DF88EC7CDF81E07ADF8E2D78DF5C
:1001B0008D2D76DF93DF6DDF88EC72DF87E070DFF7
:1001C0008C2F6EDF8BDFCF911F910F91FF90EF90FF
:1001D000DF9008951F93CF93C82F162F88DF8117C4
:1001E00031F0E199FECFCEBB1DBBE29AE19ACF91EF
:1001F0001F910895CFE9D0E0DEBFCDBFF8948AE12A
:1002000088BB81E087BB80E385BF80E48BBF1FBCD8
:1002100085E083BF8BE382BF82B78D30E8F3C09A5D
:1002200038DF8FEF3DDF35DF59DF33DF88EC38DF34
:1002300080E036DFC4E1D0E01DE0FD2FEC2FC89553
:10024000802D2EDF1150219617FFF7CF47DF21DFDA
:1002500088EC26DF80E024DF89E122DF3FDF81E0D8
:1002600046DF182F8C3108F010E0812F48DF61DF66
:10027000B19BFECF12BE82B78431E8F380E48ABF1F
:100280007894889582B78431E0F382B7883C78F41B
:100290001F5F1C3108F010E0812F31DFFFEF8F3F2F
:1002A0009F0719F410E0812F2ADF43DFEACF612F87
:1002B00081E090DFF894C098A8958895FDCF982F9D
:1002C000BB98C39AC498BC9A80E027E0BC98C49AB3
:1002D000B49BFECF880FB3998160C498BC9A21501B
:1002E00027FFF4CF992339F0C498BC9ABC98C49ADC
:1002F000BB98C39A06C0C398BB9AC498BC9ABC98D2
:10030000C49AC498BC9ABB98C39A99270895FF27AA
:10031000EE27BB27AA2760FF04C0A20FB31FE41F6C
:10032000F51F220F331F441F551F9695879577950C
:10033000679589F70097760771F79F2F8E2F7B2F90
:060340006A2F0895FFCFB3
:00000001FF
